:100000008C019D018F019001910192019301940156
:1000100095019601980199019A0183161030850087
:100020000030860064002730810083128F289B01F6
:100030000C089C006D200314980203182A2803144E
:100040000130990203182A28031401309A02031878
:100050002A281B149C031C086D2003149902031802
:100060003728031401309A02031837281B149C0305
:100070001C086D2003149A02031840280314412819
:100080001B0C00349B010C089C006D20031098078A
:10009000031C5528031001309907031C5528031031
:1000A00001309A07031C55281B149C031C086D2063
:1000B00003109907031C6228031001309A07031CE0
:1000C00062281B149C031C086D2003149A07031C50
:1000D0006B2803146C281B0C003482070034003496
:1000E0000A3400340034643400340334E834003417
:1000F0002734103401348634A0340F344234403471
:1001000098349634803482073F3406345B344F345D
:1001100066346D347D3407347F346734803483161D
:1001200000308600831214308C0009308D008E015F
:1001300007309D0017200318A4288E0A8D03031D85
:100140009A2803308C02A728422003308C02093001
:100150008D0010301D079B009B031B0884000E08B8
:100160008E0180009D0301300C07031D9A2818089A
:100170008F0097018101000000009D01FF308C007D
:100180008B011030850083161830850083120F30E4
:100190001D078400000883209B00063003151D0204
:1001A000031DD3289B171B0886001D08000085002F
:1001B0000B1DDD28970A0B11E0280000000000004D
:1001C000FB309B009B0BE22800009D0A08300311C6
:1001D0001D02031DC7280000B5309B009B0BEE28B5
:1001E00000009D018C0BC728000090309B009B0BEA
:1001F000F728000000000B1D0029970A0B110329A6
:100200000000000000000301860010308500831606
:100210001030850083120B19970A0B110108990001
:1002200017089A009B019B0A851585110B1101087F
:1002300003111902031913299B0A9B099B0A1B0A24
:0402400098008F286B
:00000001FF
